:020000020000FC
:100000000C9485040C942A000C942A000C942A0069
:100010000C942D010C942A000C942A000C942A00B4
:100020000C942A000C942A000C942A000C942A00A8
:100030000C942A000C947E020C942A000C942A0042
:100040000C942A000C942A000C942A000C942A0088
:100050000C942A00189519BC0E00669C0F00098AA2
:100060001000CE8511008B90120025AB13008DD6A9
:100070001400C2131600D4631700E3C718001D4113
:100080001A00C5D01B0031781D00010101010101DA
:100090000101010101010101010202020202020249
:1000A000020202030303030303030404040404051C
:1000B0000505050606060707070708080909090ACE
:1000C0000A0B0B0C0C0D0E0E0F1010111213131443
:1000D00015161718191A1C1D1E1F21222426272940
:1000E0002B2D2F313335383A3D3F4245484C4F5246
:1000F000565A5E62676B70757A7F858B91989EA564
:10010000ADB5BDC5CED7E0EAF5FF0DC7C59A5778A6
:10011000915DC1489138FC2B3322971AAD1413100E
:10012000800CB8098F07E00592048D03C3022602F4
:10013000AB014C010201C9009C0079005E0049003E
:1001400039002C0023001B001300000000010101F6
:100150000101020202020303030303040404040571
:100160000505050606060607070707080808080923
:100170000909090A0A0A0B0B0B0B0C0C0C0D0D0DCF
:100180000E0E0E0F0F0F101010111112121213136A
:1001900014141415151616171717181819191A1AF2
:1001A0001B1B1C1C1D1D1E1E1F1F20212122222364
:1001B000232425252627272829292A2B2B2C2D2DBA
:1001C0002E2F303031323333343536373838393AF0
:1001D0003B3C3D3E3F3F4041424344454647484902
:1001E0004A4B4C4D4E5051525354555657595A5BE9
:1001F0005C5D5F60616264656668696A6C6D6E70A3
:100200007173747677787A7B7D7E80828385868829
:100210008A8B8D8E9092949597999A9C9EA0A2A479
:10022000A5A7A9ABADAFB1B3B5B7B9BBBDBFC1C38E
:10023000C5C7C9CBCED0D2D4D6D9DBDDE0E2E4E766
:10024000E9EBEEF0F3F5F7FAFCFFE0E0E0E0E0E0E8
:10025000E0E0E0E4E8ECF0F4F8FC0F930FB70F9364
:100260001F932F933F934F935F936F937F93EF93DE
:10027000FF930F921F92509178007091790075FF53
:100280000CC01091BF0043FC109544FC109546FC37
:10029000109547FC1095110F3BC0142D77FF2CC013
:1002A00076FF4091D80076FD4091D70070FF1CC0CA
:1002B0006091D500E6E2F5E1E10FF61FC895042F45
:1002C000010F102DE6E2F5E1E00FF61FC8950027BB
:1002D00010190809140F081D14F410E000E00023A1
:1002E00009F01FEF105814C0141718F01FEF105822
:1002F0000FC010E010580CC0142D70FF08C06091A2
:10030000D500E6E2F5E1E10FF61FC895102D105873
:100310006091D60070FF60E0072D73FF07C0E6E232
:10032000F1E2E00FF61FC895002D06C0E6E2FDE2FF
:10033000E00FF61FC895002D005855FD10270093BB
:10034000D9006FE71603F00172FF012F0603E00DDD
:10035000F11D8F01159507951595079578010919D8
:100360001A0913F400E010E86091DD0040918A0062
:100370005FEF541B569528E0520F651B08F460E0B0
:10038000492D5A2D3091DF002091DE00421B530B86
:1003900013F440E050E82091780024FF02C09A0155
:1003A00013C02091E0002223D1F356039001469F11
:1003B000210D381D001C08F423958894220F331F4B
:1003C0008894220F331F9901020F131F13F40FEFAC
:1003D0001FE740918A002091780024FD40918B0016
:1003E00014039001049F210D381D001C08F423956F
:1003F000920EA31E23F42FEF3FE7922EA32E3A2D49
:10040000292DE091DE00F091DF002E1B3F0B13F44D
:1004100020E030E840918A002091780024FD40914E
:100420008B0034039001249F210D381DE20FF31F30
:1004300013F4EFEFFFE7E093DE00F093DF000E2F01
:100440001F2F2091780024FF03C0E01AF10A8701D2
:10045000F80120918C002F3F29F01203F001029F38
:10046000E10DF81D939AF0589298F5BB9398939AE2
:10047000929AE5BB9398939AEFECF0E00191200EED
:100480000191301E0191401E0191500E0191601E9C
:100490000191701EE0917900E5FD21C0E2FF1FC0CF
:1004A000E0917800E1FF10E0E1FD1FEF1123B9F0CA
:1004B0000091D900010390010091CF001127300372
:1004C000110B210C311E411E0091D0003003200C75
:1004D000311C411E0091D1003003300C411C1F9093
:1004E0000F90FF91EF917F916F915F914F913F91AD
:1004F0002F911F910F910FBF0F9118950F930FB769
:100500000F930CB1579878941F930023F2F4102F97
:10051000107F103851F0103941F0103B31F0103E8F
:1005200021F010E01093600000C1109360000F7084
:1005300003950093610010917B00112329F010179F
:1005400019F010E010936000F0C0109160001038B6
:1005500019F0113839F00AC0139510936000009318
:100560006200E3C01A951093600010C0103919F0B2
:10057000113939F03BC0139510936000009362006D
:10058000D4C01A95109360000023F9F40091620022
:1005900010916500011719F41FEF10936500109179
:1005A0006400011749F4109165001F3F31F010936A
:1005B00064001FEF10936500B8C01FEF1093640034
:1005C00010E01093A000919AB0C0009363001091C6
:1005D000640010936500109162001093640011E0B4
:1005E0001093A0001093A10091989FC0103B19F0A8
:1005F000113B39F081C013951093600000936200A5
:1006000094C01A951093600010916200AF93BF934D
:10061000103320F0103418F01035D0F064C0A1EE83
:10062000B0E0A10FB81D000F0C9310531770A0E994
:10063000B0E0A10FB81D0C91A8E9B0E0A10FB81D62
:100640000C93ACE6B0E0A10FB81D10E01C9351C0B4
:100650001054183020F11770A091790006FB10306B
:1006600011F4A0F919C0113011F4A1F915C012301C
:1006700011F4A2F911C0133011F4A3F90DC0143014
:1006800011F4A4F909C0153011F4A5F905C016300C
:1006900011F4A6F901C0A7F9A09379002AC0177038
:1006A000A091780006FB103011F4A0F919C01130A8
:1006B00011F4A1F915C0123011F4A2F911C01330D0
:1006C00011F4A3F90DC0143011F4A4F909C01530C8
:1006D00011F4A5F905C0163011F4A6F901C0A7F967
:1006E000A093780006C0A1EEB0E0A10FB81D000FE6
:1006F0000C93BF91AF9119C0103E19F0113E39F023
:1007000014C0139510936000009362000EC01A95F8
:100710001093600010916200110F110F001F00581C
:10072000109366000093670000C01F910F910FBFE8
:100730000F91579A18950F9302E30A95F1F70F91CD
:10074000089527B9369A0895349BFECF349A04B1A0
:1007500015B116950795169507950895222331F042
:100760002F93159507952A95E1F72F910895442326
:1007700041F04F9336952795179507954A95D1F7F0
:100780004F910895442341F04F93000F111F221FF2
:10079000331F4A95D1F74F910895019F8001089525
:1007A000379FE001279FA001179FD001079F902D41
:1007B000A10DB41FC51FD81D369FA001169F900D17
:1007C000A11DB41FC51FD81D269FA001069F802D07
:1007D000910DA41FB51FC81DD81D0A2F1B2F2C2F2C
:1007E0003D2F0895EE0FF0E0BB96EE0FFF1F059131
:1007F00015912591359108956F937F93E72FF2DF3F
:10080000802F912FA22FB32FE72FE395EBDF081B4B
:10081000190B2A0B3B0B8F939F93AF93BF93762FAC
:1008200060E04F93BDDF4F91BF91AF919F918F914A
:10083000080F191F2A1F3B1F7F916F91089540E0F9
:1008400002C07C5043957C30E0F70895EE0FFF1F07
:10085000E00FF81D04910895E00FF81DEE0FFF1F43
:10086000259134910895069506950695E5E8F0E002
:10087000F3DF00271127089560E0702F703718F01C
:10088000703938F00CC000E010E221E0E0E0F0E068
:100890000BC008E011E220E0ECE8FFE605C007EB42
:1008A0001DE121E0E7E6F2EE30E07ADF0E0F1F1FD8
:1008B0000895E199FECF2FBB1EBB0DBBE29AE19AD2
:1008C0000895E199FECF2FBB1EBBE09A0DB30895AA
:1008D000CCE6D0E0C40FD81D288120FD14C0302FF5
:1008E000C8E9D0E0C40FD81D1881311B0AF4319536
:1008F000353038F02160CCE6D0E0C40FD81D288315
:1009000002C010E0089511E00895F89400913400B9
:10091000006804BF04BF0FE518E00DBF1EBF8824A8
:100920002224332444245524662477249924AA2499
:1009300022273327EE27FF2705E00093CE0000E0B3
:10094000009368000093DA000093A0000093A100D8
:1009500000938C000093A9000093AA000093AB00C1
:1009600000938E0000938600009387000093880018
:1009700000936600009367000093E2000093E0009C
:1009800002E0009389000FEF00936A0000936B0070
:1009900000938A0000938B0000936400009365002D
:1009A0000EE514EB26E70093BD001093BE002093E4
:1009B000BF0000E010E020E00093C0001093C100F1
:1009C0002093C2000FEF1FEF2FEF0093C30010938F
:1009D000C4002093C50024E10093C6001093C70013
:1009E0002093C80024E60093C9001093CA00209306
:1009F000CB0000E000936C0000936D0000936E004C
:100A000000936F00009370000093710000937200D8
:100A1000009373000093B1000093B6000093A80008
:100A200000937C0000937D00009369003FB7F89429
:100A300020E010E046DF00931B01139542DF009396
:100A40001C0113953EDF00931D0113953ADF0093BF
:100A50001E01139536DF00931301139532DF0093C7
:100A6000140113952EDF0093150113952ADF0093CF
:100A700016013FBF00E00BBB00E00ABB0FEF08BB55
:100A800000E007BB00E005BB0FEF04BB0CEF02BBAF
:100A90000EEF01BB919A939A929800E003BF04E095
:100AA0000EBD06E303BD0AE005BD00E000BD0FE199
:100AB00009B900E90AB906E806B900E809BF78945F
:100AC00020918E003EDEC0E9D0E0C20FD81D3CDE92
:100AD0000883239536DEC39537DE0883239531DE00
:100AE000C39532DE088323952CDEC3952DDE088363
:100AF000239527DEC39528DE0883239522DEC39540
:100B000023DE088323951DDEC3951EDE088323950F
:100B100018DEC39519DE088320E020938E0011DED5
:100B200000919000009398000093110100919100B2
:100B300000939900009312010091920000939A0093
:100B40000091930000939B000091940000939C00FF
:100B50000091950000939D000091960000939E00E7
:100B6000009317010091970000939F0000931801D4
:100B70000CB51DB50093A2001093A3000CB51DB5D4
:100B80002091A2003091A300021B130B0A561841BA
:100B900008F4EEC00CB51DB50093A2001093A3009D
:100BA00000E111E020E130E040E050E0E2B3E06F2E
:100BB000E027E2BBC0DDE6B3E0FF312BE1FF322BE3
:100BC000E2FF412BE3FF422BE4FF512B110F220FD9
:100BD000000F61F702B3006F02BB309374004093C3
:100BE000750050937A0010916B0010FF08C030938D
:100BF000760040937700309378004093790000911D
:100C0000740010917600011739F1209178001027B7
:100C100010FF02C000FB20F911FF02C001FB21F907
:100C200012FF02C002FB22F913FF02C003FB23F9EB
:100C300014FF02C004FB24F915FF02C005FB25F9CF
:100C400016FF02C006FB26F917FF02C007FB27F9B3
:100C50002093780020937600009175001091770022
:100C6000011739F120917900102710FF02C000FB15
:100C700020F911FF02C001FB21F912FF02C002FBA3
:100C800022F913FF02C003FB23F914FF02C004FB87
:100C900024F915FF02C005FB25F916FF02C006FB6B
:100CA00026F917FF02C007FB27F92093790020934C
:100CB000770000917A0000937B00309178001091CA
:100CC0006B0010FF0AC030FF00E030FD01E0009330
:100CD0006A00112710936B004BC030FF00E030FD1D
:100CE00001E010916A00011709F442C000936A0004
:100CF00030FD07C001E00093DB0000E00093DC0062
:100D000006C000E00093DB0004E00093DC00002755
:100D100000936C0000936D0000936E0000936F00D1
:100D200000937000009371000093720000937300B1
:100D30000091900000939800009191000093990019
:100D40000091920000939A000091930000939B0001
:100D50000091940000939C000091950000939D00E9
:100D60000091960000939E000091970000939F00D1
:100D70000091DB0007FD43C0E19941C000FD14C0B4
:100D80000091DC00053039F0063041F0073049F0C1
:100D9000109113011DC0109114011AC0109115017A
:100DA00017C01091160114C00091DC00013039F019
:100DB000023041F0033049F010911B0109C010913D
:100DC0001C0106C010911D0103C010911E0100C03E
:100DD00030E03FBB0EBB1DBB3FB7F894E29AE19AEF
:100DE0003FBF033031F0073021F003950093DC0062
:100DF00006C010E01093DC001FEF1093DB00A4DCB2
:100E000020918E0020938F00C0E9D0E0C20FD81D42
:100E100008832395277020938E0093DC40918F00E8
:100E2000403069F455DD112311F000931101009158
:100E300011010C3F08F00CEF00931101A2C04130EA
:100E400031F446DD112341F1009312019AC046307E
:100E500099F43EDD112311F0009317010091170161
:100E60000695025110F404E004C0043008F001C0FB
:100E700004E00093D80085C0473079F429DD1123C0
:100E800011F00093180100911801F6DC105800933E
:100E90007C0010937D0075C074C03091780030FDE7
:100EA0000C947807423031F413DD112341F10093A3
:100EB000130125C0433041F40BDD1123C1F0009331
:100EC0006900009314015DC0443031F401DD112349
:100ED000D9F10093150138C0453049F4F9DC1123EC
:100EE00031F00695102F1695010F0093160149C099
:100EF0004230D9F4EDDC112311F000931B01009175
:100F00001B013091790034FF08C03FEF309384001B
:100F1000309383000093850034C030E03093840028
:100F200000938300009385002CC0433031F4D0DC63
:100F3000112339F100931C0124C04430D9F4C8DCDA
:100F4000112311F000931D0100911D0130917900D2
:100F500034FF08C03FEF3093800030937F00009350
:100F600081000FC030E03093800000937F00009339
:100F7000810007C0453029F4ABDC112311F0009348
:100F80001E0100916300000F10911501019F109246
:100F9000B0006CB57DB5262F372F0091A4001091BD
:100FA000A500601B710B2093A4003093A5006093F3
:100FB000A6007093A70000911301009554DC609186
:100FC000A6007091A700ECDB3091B2004091B30015
:100FD0005091B4005058F0E0E091B100EE23A1F43C
:100FE0006091C3007091C4008091C500300F411F13
:100FF000521F20F0361747075807C8F0362F472FE3
:10100000582FE1E0F1E013C06091C0007091C10081
:101010008091C200301B410B520B20F06317740704
:10102000850728F0362F472F582FE0E0F1E0E093B6
:10103000B10050583093B2004093B3005093B400C5
:1010400000E010E020E0E0917800E2FF09C0FF231B
:10105000B1F00091BD001091BE002091BF002F772C
:101060000093C0001093C1002093C200009510951A
:1010700020950093C3001093C4002093C5000091F5
:10108000780002FF05C0FF2361F05091BF0007C048
:101090000091780003FF03C0550F5FE7581D509380
:1010A000B500009114011091E200011708F4012F1E
:1010B0000093690000911701069506950095D3DB12
:1010C0006091A6007091A7006BDB3091B700409152
:1010D000B8005091B9005058F0E0E091B600EE230E
:1010E000A1F46091C9007091CA008091CB00300FCB
:1010F000411F521F20F0361747075807C8F0362FF8
:10110000472F582FE1E0F1E013C06091C6007091C5
:10111000C7008091C800301B410B520B20F06317B1
:101120007407850728F0362F472F582FE0E0F1E0AD
:10113000E093B60050583093B7004093B8005093F6
:10114000B90050585093D7001091A80000911E018B
:10115000113069F000917F00123049F00091810058
:10116000143029F060918000133039F13AC07BDBF4
:101170006091A6007091A70013DB3091A900409107
:10118000AA005091AB006091A8006430D1F06230A9
:1011900049F0300F411F521FF0F43FEF4FEF5FEF68
:1011A00002E017C0301B410B520B78F060918000B9
:1011B000651788F003E00093A80033274427562FD3
:1011C0000AC0301B410B520B30F430E040E050E0DD
:1011D00000E00093A8003093A9004093AA00509328
:1011E000AB001091AC0000911C01113069F000912E
:1011F0008300123049F000918500143029F060918D
:101200008400133039F13CC02EDB6091A600709150
:10121000A700C6DA3091AD004091AE005091AF000A
:101220006091AC006430D1F0623049F0300F411F62
:10123000521F00F53FEF4FEF5FEF02E019C0301B88
:10124000410B520B78F060918400651798F003E031
:101250000093AC0033274427562F0CC0301B410BA2
:10126000520B40F430E040E050E000E00093E0003A
:101270000093AC003093AD004093AE005093AF00AC
:101280000091A000002371F404E01091A800112344
:1012900051F10093A8001091AC00112321F10093AB
:1012A000AC0021C00091A1000023E9F000E0009310
:1012B000A10000918900002319F00A95009389008C
:1012C00001E00093A8000093AC000093E0000FEF52
:1012D0001FEF2FE70093B2001093B3002093B400E8
:1012E00001E00093B10090E060E0709164007F3F06
:1012F00011F4AEC07C507136E8F701C0745F7432EF
:10130000E8F37C5090918600A0918700B09188000E
:1013100000918900002381F500911601A4DA6F93F2
:101320007F93622F732F00E010E02091A600309190
:10133000A70043E01CDA34DA7F916F91302F412F00
:10134000522F90918600A0918700B09188006A1773
:101350007B0738F4931BA40BB50B6A177B0750F07F
:1013600006C0930FA41FB51F6A177B0718F490E0FF
:10137000A62FB72F6A2F7B2F90938600609387004C
:1013800070938800009166001091670025E0E6D90F
:10139000202F312F020F131F020F131F600F711F19
:1013A00070938D000091780007FF0C94F409009170
:1013B000B500109169002091780026FF10E0212FE0
:1013C0001695203810F01058120F0103800124E008
:1013D000C5D9600F711F77231AF460E070E004C074
:1013E0007D3610F060E07CE66F937F93972F9D50E1
:1013F00008F499279695969596959093D5001FDABF
:10140000FBD9C0D91093CF002093D0003093D100E6
:101410007F916F9100917C0010917D0024E09ED916
:10142000600F711F0091790001FD745F972F9D502F
:1014300008F499279695969596959093D600FFD99E
:10144000DBD9A0D91093D2002093D3003093D400DD
:10145000E0E0F0E00091780007FD0DC00091B500DC
:10146000109169002091780026FF10E00103E12D22
:10147000F0E0111CFF0B0091AF001091B000019F34
:101480008001001FE11FF81D00918D00000F005624
:101490001BEA0103800120E017FD2FEFE10FF21F8F
:1014A0000091120111270E0F1F1F112312F400E0EB
:1014B00002C009F00FEF0695E5E4F0E0C7D900930C
:1014C0008A000A5008F400E000938B00109111018B
:1014D00000918A00003110F0012F06C0E5E2F1E032
:1014E000B5D9011708F0012F0093DD000091AB0082
:1014F000E5EAF0E0ABD900938C000091BD001091BB
:10150000BE002091BF0027FB30F922FB40F93427B1
:101510003695001F111F221F0093BD001093BE00BF
:101520002093BF002BCB801211151616161819190F
:101530001A1B1C1D1E1F202021222324252627279D
:1015400028292A2B2C2D2D2E2F30313233343435AF
:10155000363738393A3A3B3C3D3E3F4041414243C1
:10156000444546474748494A4B4C4D4D4E4F5051D4
:10157000525353545556575859595A5B5C5D5E5FE8
:101580006060616263646566666768696A6B6C6DFA
:101590006D6E6F70717273737475767778797A7A0D
:1015A0007B7C7D7E7F808080818283848586868728
:1015B00088898A8B8C8D8D8E8F9091929393949540
:1015C000969798999A9A9B9C9D9E9FA0A0A1A2A352
:1015D000A4A5A6A7A7A8A9AAABACADADAEAFB0B164
:1015E000B2B3B3B4B5B6B7B8B9B9BABBBCBDBEBF78
:1015F000BFC0C1C2C3C4C5C6C6C7C8C9CACBCCCC8C
:10160000CDCECFD0D1D2D3D3D4D5D6D7D8D9D9DA9D
:10161000DBDCDDDEDFE0E0E1E2E3E4E5E6E7E7E8AE
:10162000EAEAEAEBEFEE80111015171516191919F1
:101630001A1C1C1D1E1F1F2022222324252626279C
:1016400028292A2B2C2C2D2E2F30313233333435B0
:1016500036373839393A3B3C3D3E3F4040414243C2
:10166000444546464748494A4B4C4C4D4E4F5051D5
:10167000525353545556575859595A5B5C5D5E5FE7
:101680006060616263646566666768696A6B6C6DF9
:101690006D6E6F70717273737475767778797A7A0C
:1016A0007B7C7D7E7F808080818283848586868727
:1016B00088898A8B8C8D8D8E8F909192939394953F
:1016C000969798999A9A9B9C9D9E9FA0A0A1A2A351
:1016D000A4A5A6A7A7A8A9AAABACADADAEAFB0B163
:1016E000B2B3B4B4B5B6B7B8B9BABABBBCBDBEBF75
:1016F000C0C0C1C2C3C4C5C6C7C7C8C9CACBCCCD88
:10170000CDCECFD0D1D2D3D4D4D5D6D7D8D9DADA9A
:10171000DBDCDDDEDEE0E1E1E2E3E4E4E6E7E7E7AF
:10172000EAEBE9EBF0EF801C161414141516181AE6
:101730001B1C1D1D1E1E1F2021222324252627279A
:101740002829292A2B2C2D2E2F30313232333435B3
:10175000363738393A3A3B3C3D3E3E3F40414243C2
:10176000444546464748494A4B4C4D4D4E4F5051D3
:10177000525253545556575859595A5B5C5D5E5FE7
:101780006061616263646565666768696A6B6C6DF8
:101790006D6E6F7071727374747576777879797A0B
:1017A0007B7C7D7E7F808080818283848586878725
:1017B00088898A8B8C8C8D8E8F909192939394953F
:1017C000969798999A9B9B9C9D9E9F9FA0A1A2A350
:1017D000A4A5A6A7A7A8A9AAABACADAEAEAFB0B161
:1017E000B2B3B3B4B5B6B7B8B9BABABBBCBDBEBF75
:1017F000C0C1C2C2C3C4C5C6C6C7C8C9CACBCCCD86
:10180000CECECFD0D1D2D3D4D5D6D7D7D8D9D9DA96
:10181000DBDCDDDEDFE0E1E2E2E3E3E4E5E6E8EAAB
:10182000EBECECECEAE4800A0F1A15131919171AFD
:101830001C1A1C1E1D1E2120212323232526262899
:1018400029292A2C2C2C2E2E2F30313133343435AB
:10185000373738393A3A3C3C3D3E3F3F41424243BC
:10186000444546474748494A4B4C4D4D4E505051D0
:101870005253535555565758595A5B5B5C5D5E5FE2
:101880006061616263646566666769696A6B6C6CF6
:101890006E6E6F70717273747475767778797A7A08
:1018A0007B7C7D7E7F7F8081818283848586868725
:1018B00088898A8B8C8C8D8E8F909192929494953E
:1018C000969797999A9A9B9C9D9E9F9FA0A1A2A351
:1018D000A4A5A5A6A7A8A9AAABABADADAEAFB0B065
:1018E000B2B3B3B4B5B6B7B8B9B9BABBBCBDBEBE76
:1018F000BFC1C1C2C3C4C4C6C6C7C8C9C9CBCCCC8A
:10190000CDCFCFD0D1D2D2D4D4D4D6D7D7D8DADA9B
:10191000DBDDDDDDDFE0DFE2E3E2E4E6E4E6E9E7AC
:10192000E7EDEBE6F1F680011B131519141C161CEC
:10193000191C1D1C201D211F222223252427262897
:1019400028292B2A2D2C2E2E3030313232343436A9
:10195000363738383A3A3C3C3D3E3F4040424243BD
:101960004445464648484A4A4B4C4C4E4E505051CE
:101970005253545456565758595A5A5C5C5D5E5FE0
:1019800060606262636465666668686A6A6B6C6DF3
:101990006E6E7070717273747476767778797A7A05
:1019A0007C7C7D7E7F808080818283848486868724
:1019B00088898A8A8C8C8D8E8F9090929293949540
:1019C000969698989A9A9B9C9D9E9EA0A0A1A2A351
:1019D000A4A4A6A6A7A8A9AAAAACACADAEAFB0B065
:1019E000B2B2B4B4B5B6B6B8B8BABABBBCBDBEBE76
:1019F000C0C0C1C2C3C4C4C6C6C8C8C9CACACCCC88
:101A0000CECECFD0D0D2D2D4D3D6D5D7D8D8DAD99B
:101A1000DCDBDDDEDEE1DFE3E0E4E3E4E7E4EAE4AF
:101A2000ECE7EBEDE5FF801A01181E11131D1B15E5
:101A30001A1F1B1A20211E1F242321242725252994
:101A400029282A2C2C2B2E2F2E2F323232333535AB
:101A500035383938393B3C3B3D3F3E3F41424243BC
:101A6000454545474848494B4B4B4D4E4E4F5051CD
:101A70005152545555565858585A5B5B5C5E5E5EE1
:101A80006061616264646466676768696A6B6B6DF4
:101A90006E6E6F71717173747475777777797A7A06
:101AA0007B7D7D7D7F808080818383838586868723
:101AB0008989898B8C8C8D8F8F8F9192929395953C
:101AC00096979899999A9C9C9C9E9F9FA0A2A2A24F
:101AD000A4A5A5A6A8A8A8AAABABACAEAFAFB0B161
:101AE000B2B2B3B5B5B5B7B8B8B9BBBBBBBDBEBE76
:101AF000BFC1C2C1C3C5C4C5C7C8C7C8CBCBCBCD86
:101B0000CECECED1D2D1D2D5D4D4D6D8D7D7DBDB96
:101B1000D9DCDFDDDCE1E2DFE0E6E5E1E6EBE5E3B1
:101B2000EDEFE2E8FFE680390B000D1D211B1313DA
:101B30001920211D1A1B2024242120222628282692
:101B400026282B2D2C2B2B2E3132313031343636AA
:101B5000353537393B3B3A3B3C3F40403F404244C0
:101B60004545454547494A4A4A4B4D4E4F4F4F50D0
:101B7000525454545456585959595A5B5D5E5E5EDE
:101B80005F61626363636466676868686A6C6C6DF2
:101B90006D6E6F71717272737576777777787A7B05
:101BA0007C7C7C7E7F808080818284848485868822
:101BB0008989898A8B8D8E8E8F8F9192939394943D
:101BC00096989898999A9C9D9D9D9E9FA1A2A2A24D
:101BD000A3A5A6A7A7A7A8AAACACACACAEB0B1B160
:101BE000B1B2B3B5B6B6B6B7B9BBBBBBBBBCBEC072
:101BF000C1C0C0C1C4C5C6C5C5C7C9CBCBCACACC84
:101C0000CFD0CFCECFD2D5D5D4D3D5D8DADAD8D895
:101C1000DADEE0DFDCDCE0E5E6E3DFE0E7EDEDE5A2
:101C2000DFE3F3FFF5C78051290E02030C172024D0
:101C3000221D1815161A20242626242120212428A6
:101C40002B2C2C2B2A292A2C2F32333333323132AE
:101C50003437393B3B3A3A3A3B3D3F4142424242BC
:101C600042434547494A4A4A4A4A4B4C4E505152D0
:101C700052515253545658595A59595A5B5C5E60E6
:101C800061616161626364666869696969696A6CF6
:101C90006E6F707171717172747677787979797904
:101CA0007A7C7D7F8080808080818384868787871F
:101CB0008788898A8C8E8F8F8F8F90919294969738
:101CC00097979797989A9C9D9E9F9F9F9FA0A2A44D
:101CD000A5A6A7A7A6A7A8AAACADAEAFAEAEAFB05B
:101CE000B2B4B5B6B6B6B6B6B7B9BBBDBEBEBEBE6B
:101CF000BEBFC1C3C5C6C6C6C5C5C7C9CCCECFCE7B
:101D0000CDCDCDCED1D4D6D7D6D5D4D4D5D8DCDF91
:101D1000E0DFDCDADADCE0E6EAEBE8E3DEDCE0E9AF
:101D2000F4FDFEF2D7AF8061442B180B0403060CC0
:101D3000141C2226282725221E1C1B1B1D2124289B
:101D40002B2E2F2F2E2C2B2A2A2B2C2F31343638AA
:101D500039393938373737383A3C3E4042444445C0
:101D600044444444444547484A4C4E4F50505050D8
:101D700050505152535557595A5B5C5C5C5C5C5CEB
:101D80005D5E606163656667686868686869696BFD
:101D90006C6E707173747474747475757677797A07
:101DA0007C7E7F808080808080808182848687891D
:101DB0008A8B8B8C8C8C8C8C8D8F90929495979732
:101DC0009898989898999A9B9D9FA0A2A3A4A4A440
:101DD000A4A4A4A5A6A7A9ABADAEAFB0B0B0B0B057
:101DE000B0B1B2B4B6B8B9BBBCBCBCBCBCBBBCBC6B
:101DF000BEC0C2C4C6C8C9C9C9C8C7C7C7C8CACC7B
:101E0000CFD1D4D5D6D6D5D4D2D1D1D2D5D8DCDF86
:101E1000E3E5E5E4E2DEDBD9D8DADEE4ECF4FAFD72
:101E2000FCF5E8D5BC9F806D5A49382A1E140C0871
:101E3000050506090D12181D22262A2C2E2F2E2DDF
:101E40002C2A2927262524252627292C2F313437EB
:101E5000393B3C3D3D3D3D3D3C3B3B3B3B3B3C3DC5
:101E60003F41434547494B4D4E4F4F505050504FC7
:101E70004F4F4F505052535456585A5C5E5F6062F9
:101E800062636363636363636364646567686A6B07
:101E90006D6F7172747575767677777777777777F8
:101EA00078797A7B7D7F8081838586878889898917
:101EB000898989898A8A8B8B8C8E8F919395969844
:101EC000999B9C9C9D9D9D9D9D9D9D9D9E9EA0A141
:101ED000A2A4A6A8AAACADAEB0B0B1B1B1B1B0B039
:101EE000B0B0B1B1B2B3B5B7B9BBBDBFC1C3C4C562
:101EF000C5C5C5C5C4C3C3C3C3C3C4C5C7C9CCCF87
:101F0000D1D4D7D9DADBDCDBDAD9D7D6D4D3D2D166
:101F1000D2D4D6DADEE3E8EEF3F7FAFBFBF8F4EC22
:101F2000E2D6C8B7A6938074685B50453A31282042
:101F30001A140F0C0A080808090B0E1114181C209B
:101F400023272A2E30333536383839393838373662
:101F500036353433323232323333343537393B3D30
:101F60003F414345484A4C4D4F50515253535353B0
:101F70005353535353525252535354545556585922
:101F80005B5C5E6062646667696B6C6D6E6F7070DF
:101F90007171717171717171717272727374747621
:101FA00077787A7B7D7F808183858688898A8C8C0F
:101FB0008D8E8E8E8F8F8F8F8F8F8F8F8F90909132
:101FC0009293949597999A9C9EA0A2A4A5A7A8AA3B
:101FD000ABACACADADAEAEAEADADADADADADADAD32
:101FE000ADAEAFB0B1B3B4B6B8BBBDBFC1C3C5C76A
:101FF000C9CBCCCDCDCECECECECDCCCBCACAC9C826
:10200000C8C7C7C8C8CACBCDD0D2D6D9DDE0E4E8AE
:10201000ECEFF2F5F7F8F8F8F6F4F1ECE6E0D8CFEB
:10202000C6BBB0A5988C80776E655D544C443C353A
:102030002F29231E1A1613100E0C0B0B0B0B0C0E54
:10204000101214171A1D202326292C2F3235373A47
:102050003C3D3F4042434344444444444443434260
:102060004241414140404040404141424344454655
:1020700048494B4D4F51535557595B5C5E60626305
:102080006566676869696A6B6B6B6B6B6C6C6B6BB5
:102090006B6B6B6C6C6C6C6D6D6E6F70717273755D
:1020A0007678797B7D7F8081838587888A8B8D8E0A
:1020B0008F909192939394949494959595959594EB
:1020C00094959595959596979798999A9B9D9EA08E
:1020D000A2A4A5A7A9ABADAFB1B3B5B7B8BABBBC05
:1020E000BDBEBFBFC0C0C0C0C0BFBFBFBEBEBDBD04
:1020F000BCBCBCBCBCBCBDBDBEC0C1C3C4C6C9CBDE
:10210000CED1D4D7DADDE0E3E6E9ECEEF0F2F4F597
:10211000F5F5F5F4F2F0EDEAE6E2DDD7D1CBC4BC9B
:10212000B4ACA39B928980E6E7E5E4E5E6E5E5E566
:10213000E5E5E5E5E5E5E5E5E5E5E5E5E5E5E5E54F
:10214000E5E5E5E5E5E5E5E5E5E5E5E5E5E5E5E53F
:10215000E5E5E5E5E5E5E5E5E5E5E5E5E5E5E5E52F
:10216000E5E5E5E5E5E5E5E5E5E5E5E5E5E5E5E51F
:10217000E5E5E5E5E5E5E5E5E5E5E5E5E5E5E5E50F
:10218000E5E5E5E5E5E5E5E5E5E5E5E5E5E5E5E5FF
:10219000E5E5E5E5E5E5E5E5E5E5E5E5E5E5E5E5EF
:1021A000E6E5E4E5E7E6801A191B1C1B1A1B1B1B5E
:1021B0001B1B1B1B1B1B1B1B1B1B1B1B1B1B1B1B6F
:1021C0001B1B1B1B1B1B1B1B1B1B1B1B1B1B1B1B5F
:1021D0001B1B1B1B1B1B1B1B1B1B1B1B1B1B1B1B4F
:1021E0001B1B1B1B1B1B1B1B1B1B1B1B1B1B1B1B3F
:1021F0001B1B1B1B1B1B1B1B1B1B1B1B1B1B1B1B2F
:102200001B1B1B1B1B1B1B1B1B1B1B1B1B1B1B1B1E
:102210001B1B1B1B1B1B1B1B1B1B1B1B1B1B1B1B0E
:102220001A1B1C1B191A80E6E8E4E4E6E6E4E5E67E
:10223000E5E4E5E5E5E5E5E5E5E5E5E5E5E5E5E54F
:10224000E5E5E5E5E5E5E5E5E5E5E5E5E5E5E5E53E
:10225000E5E5E5E5E5E5E5E5E5E5E5E5E5E5E5E52E
:10226000E5E5E5E5E5E5E5E5E5E5E5E5E5E5E5E51E
:10227000E5E5E5E5E5E5E5E5E5E5E5E5E5E5E5E50E
:10228000E5E5E5E5E5E5E5E5E5E5E5E5E5E5E5E5FE
:10229000E5E5E5E5E5E5E5E5E5E5E5E4E5E6E5E4EF
:1022A000E6E6E4E4E8E6801A181C1C1A1A1C1B1A5D
:1022B0001B1C1B1B1B1B1B1B1B1B1B1B1B1B1B1B6D
:1022C0001B1B1B1B1B1B1B1B1B1B1B1B1B1B1B1B5E
:1022D0001B1B1B1B1B1B1B1B1B1B1B1B1B1B1B1B4E
:1022E0001B1B1B1B1B1B1B1B1B1B1B1B1B1B1B1B3E
:1022F0001B1B1B1B1B1B1B1B1B1B1B1B1B1B1B1B2E
:102300001B1B1B1B1B1B1B1B1B1B1B1B1B1B1B1B1D
:102310001B1B1B1B1B1B1B1B1B1B1B1C1B1A1B1C0C
:102320001A1A1C1C181A80DDE3E5E6E7E7E6E6E585
:10233000E5E4E4E5E5E5E6E6E6E6E5E5E5E5E5E54B
:10234000E5E5E5E6E5E5E5E5E5E5E5E5E5E5E5E53C
:10235000E5E5E5E5E5E5E5E5E5E5E5E5E5E5E5E52D
:10236000E5E5E5E5E5E5E5E5E5E5E5E5E5E5E5E51D
:10237000E5E5E5E5E5E5E5E5E5E5E5E5E5E5E5E50D
:10238000E5E5E5E5E5E5E5E5E5E6E5E5E5E5E5E5FC
:10239000E5E5E5E6E6E6E6E5E5E5E4E4E5E5E6E6E9
:1023A000E7E7E6E5E3DD80231D1B1A19191A1A1B5E
:1023B0001B1C1C1B1B1B1A1A1A1A1B1B1B1B1B1B6F
:1023C0001B1B1B1A1B1B1B1B1B1B1B1B1B1B1B1B5E
:1023D0001B1B1B1B1B1B1B1B1B1B1B1B1B1B1B1B4D
:1023E0001B1B1B1B1B1B1B1B1B1B1B1B1B1B1B1B3D
:1023F0001B1B1B1B1B1B1B1B1B1B1B1B1B1B1B1B2D
:102400001B1B1B1B1B1B1B1B1B1A1B1B1B1B1B1B1D
:102410001B1B1B1A1A1A1A1B1B1B1C1C1B1B1A1A10
:1024200019191A1B1D2380EDEAE0E5E8E3E4E7E46F
:10243000E4E6E5E4E6E5E4E5E6E4E5E6E4E5E6E54C
:10244000E5E5E5E4E5E5E4E5E5E4E5E5E5E5E5E53F
:10245000E5E5E5E5E5E5E5E5E5E5E5E5E5E5E5E52C
:10246000E5E5E5E5E5E5E5E5E5E5E5E5E5E5E5E51C
:10247000E5E5E5E5E5E5E5E5E5E5E5E5E5E5E5E50C
:10248000E5E5E5E4E5E5E4E5E5E4E5E5E5E5E6E5FE
:10249000E4E6E5E4E6E5E4E5E6E4E5E6E4E4E7E4ED
:1024A000E3E8E5E0EAED801316201B181D1C191C5B
:1024B0001C1A1B1C1A1B1C1B1A1C1B1A1C1B1A1B6C
:1024C0001B1B1B1C1B1B1C1B1B1C1B1B1B1B1B1B59
:1024D0001B1B1B1B1B1B1B1B1B1B1B1B1B1B1B1B4C
:1024E0001B1B1B1B1B1B1B1B1B1B1B1B1B1B1B1B3C
:1024F0001B1B1B1B1B1B1B1B1B1B1B1B1B1B1B1B2C
:102500001B1B1B1C1B1B1C1B1B1C1B1B1B1B1A1B19
:102510001C1A1B1C1A1B1C1B1A1C1B1A1C1C191C0A
:102520001D181B20161380F5DFE6E7E2E8E1E8E37B
:10253000E5E5E4E7E3E6E4E5E5E4E6E4E6E4E5E54D
:10254000E4E6E4E6E4E5E5E5E5E4E6E4E5E5E5E53D
:10255000E4E6E4E5E5E5E5E4E5E4E5E5E5E5E4E52F
:10256000E4E5E5E5E5E4E5E4E5E5E5E5E4E5E4E520
:10257000E5E5E5E4E5E4E5E5E5E5E4E6E4E5E5E50E
:10258000E5E4E6E4E5E5E5E5E4E6E4E6E4E5E5E4FE
:10259000E6E4E6E4E5E5E4E6E3E7E4E5E5E3E8E1EF
:1025A000E8E2E7E6DFF5800B211A191E181F181D57
:1025B0001B1B1C191D1A1C1B1B1C1A1C1A1C1B1B69
:1025C0001C1A1C1A1C1B1B1B1B1C1A1C1B1B1B1B59
:1025D0001C1A1C1B1B1B1B1C1B1C1B1B1B1B1C1B47
:1025E0001C1B1B1B1B1C1B1C1B1B1B1B1C1B1C1B36
:1025F0001B1B1B1C1B1C1B1B1B1B1C1A1C1B1B1B28
:102600001B1C1A1C1B1B1B1B1C1A1C1A1C1B1B1C17
:102610001A1C1A1C1B1B1C1A1D191C1B1B1D181F06
:10262000181E191A210B80DEF6E2DDE9E9E1E3E983
:10263000E6E2E5E8E4E3E7E6E3E4E7E5E3E5E7E44B
:10264000E4E6E6E4E5E6E5E4E5E6E4E4E6E6E4E53A
:10265000E6E5E4E5E6E4E4E6E5E4E5E6E5E4E5E62A
:10266000E4E4E6E5E4E5E6E5E4E5E6E4E4E6E5E41D
:10267000E5E6E5E4E5E6E4E4E6E5E4E5E6E5E4E60A
:10268000E6E4E4E6E5E4E5E6E5E4E6E6E4E4E7E5F9
:10269000E3E5E7E4E3E6E7E3E4E8E5E2E6E9E3E1EE
:1026A000E9E9DDE2F6DE80220A1E2317171F1D1757
:1026B0001A1E1B181C1D191A1D1C191B1D1B191C69
:1026C0001C1A1A1C1B1A1B1C1B1A1C1C1A1A1C1B5A
:1026D0001A1B1C1B1A1C1C1A1B1C1B1A1B1C1B1A4A
:1026E0001C1C1A1B1C1B1A1B1C1B1A1C1C1A1B1C37
:1026F0001B1A1B1C1B1A1C1C1A1B1C1B1A1B1C1A2A
:102700001A1C1C1A1B1C1B1A1B1C1A1A1C1C191B1A
:102710001D1B191C1D1A191D1C181B1E1A171D1F05
:102720001717231E0A2280C1ECF7EDDFDBE2EAEC8B
:10273000E7E1E0E4E9E9E5E2E2E5E8E8E5E3E3E64C
:10274000E8E7E4E3E4E6E7E6E4E3E4E6E7E6E4E337
:10275000E5E6E7E5E4E4E5E7E6E5E4E4E5E7E6E524
:10276000E4E4E6E7E6E4E4E4E6E7E6E4E4E5E6E715
:10277000E5E4E4E5E6E7E5E4E4E5E7E6E5E3E4E609
:10278000E7E6E4E3E4E6E7E6E4E3E4E7E8E6E3E3F8
:10279000E5E8E8E5E2E2E5E9E9E4E0E1E7ECEAE2E0
:1027A000DBDFEDF7ECC1803F14091321251E161461
:1027B000191F201C17171B1E1E1B18181B1D1D1A66
:1027C00018191C1D1C1A191A1C1D1C1A191A1C1D5B
:1027D0001B1A191B1C1C1B191A1B1C1C1B191A1B4E
:1027E0001C1C1A191A1C1C1C1A191A1C1C1B1A193D
:1027F0001B1C1C1B1A191B1C1C1B191A1B1D1C1A29
:10280000191A1C1D1C1A191A1C1D1C19181A1D1D19
:102810001B18181B1E1E1B17171C201F1914161E11
:1028200025211309143F80ABD0E9F6F7F0E7DFDB91
:10283000DDE2E8EBECEAE6E2E0E1E3E7E9EAE9E63B
:10284000E3E2E2E4E6E8E9E8E6E4E3E3E4E6E7E835
:10285000E8E6E4E3E3E4E5E7E8E8E6E5E3E3E4E526
:10286000E7E8E8E7E5E4E3E4E5E7E8E8E7E5E4E30B
:10287000E3E5E6E8E8E7E5E4E3E3E4E6E8E8E7E6FD
:10288000E4E3E3E4E6E8E9E8E6E4E2E2E3E6E9EAF1
:10289000E9E7E3E1E0E2E6EAECEBE8E2DDDBDFE7F3
:1028A000F0F7F6E9D0AB805530170A091019212549
:1028B000231E181514161A1E201F1D191716171A75
:1028C0001D1E1E1C1A1817181A1C1D1D1C1A19185B
:1028D000181A1C1D1D1C1B1918181A1B1D1D1C1B4A
:1028E000191818191B1C1D1C1B191818191B1C1D45
:1028F0001D1B1A1818191B1C1D1D1C1A1818191A33
:102900001C1D1D1C1A1817181A1C1E1E1D1A17161E
:1029100017191D1F201E1A161415181E23252119FC
:1029200010090A173055809CB7CEE0EEF6F8F7F2A2
:10293000ECE6E1DDDCDCDFE2E6E9ECEDEDEBE9E63F
:10294000E3E1E0E0E2E3E6E8E9EAEAEAE8E6E4E334
:10295000E2E2E2E4E5E7E9E9EAE9E8E6E5E3E2E222
:10296000E3E4E5E7E8E9E9E9E8E7E5E4E3E2E2E30F
:10297000E5E6E8E9EAE9E9E7E5E4E2E2E2E3E4E6FC
:10298000E8EAEAEAE9E8E6E3E2E0E0E1E3E6E9EBE7
:10299000EDEDECE9E6E2DFDCDCDDE1E6ECF2F7F8B8
:1029A000F6EEE0CEB79C8064493220120A08090E88
:1029B000141A1F232424211E1A1714131315171A6F
:1029C0001D1F20201E1D1A1817161616181A1C1D5A
:1029D0001E1E1E1C1B1917171617181A1B1D1E1E4C
:1029E0001D1C1B191817171718191B1C1D1E1E1D3F
:1029F0001B1A1817161717191B1C1E1E1E1D1C1A32
:102A00001816161617181A1D1E20201F1D1A171526
:102A1000131314171A1E212424231F1A140E090835
:102A20000A122032496480909FAFBDCAD6E0E8EF19
:102A3000F4F7F9FAF9F7F4F1EDEAE6E3E1DEDDDCCB
:102A4000DCDDDEDFE1E4E6E8EAECEDEEEFEFEEED13
:102A5000ECEAE9E7E5E3E2E1E0E0E0E1E2E3E4E635
:102A6000E7E9EAECEDEDEDEDEDECEAE9E7E6E4E3CC
:102A7000E2E1E0E0E0E1E2E3E5E7E9EAECEDEEEFF8
:102A8000EFEEEDECEAE8E6E4E1DFDEDDDCDCDDDE06
:102A9000E1E3E6EAEDF1F4F7F9FAF9F7F4EFE8E04B
:102AA000D6CABDAF9F908070615143362A2018115D
:102AB0000C09070607090C0F13161A1D1F222324E1
:102AC000242322211F1C1A18161413121111121379
:102AD000141617191B1D1E1F2020201F1E1D1C1A37
:102AE000191716141313131313141617191A1C1D80
:102AF0001E1F2020201F1E1D1B1917161413121134
:102B00001112131416181A1C1F2122232424232205
:102B10001F1D1A16130F0C09070607090C111820A0
:102B20002A36435161708089939DA6AFB8C0C8D042
:102B3000D7DDE3E8EDF1F4F7F9FBFCFCFCFBFAF977
:102B4000F8F6F4F1EFEDEAE8E6E4E2E0DFDEDDDC02
:102B5000DCDCDCDDDDDEE0E1E2E4E6E7E9EBECEE47
:102B6000EFF0F1F2F3F3F3F3F3F2F1F0EFEEECEB5D
:102B7000E9E7E6E4E2E1E0DEDDDDDCDCDCDCDDDE55
:102B8000DFE0E2E4E6E8EAEDEFF1F4F6F8F9FAFB6B
:102B9000FCFCFCFBF9F7F4F1EDE8E3DDD7D0C8C0AD
:102BA000B8AFA69D938980776D635A5148403830FD
:102BB00029231D18130F0C09070504040405060733
:102BC000080A0C0F111316181A1C1E202122232488
:102BD000242424232322201F1E1C1A191715141223
:102BE00011100F0E0D0D0D0D0D0E0F1011121415ED
:102BF00017191A1C1E1F20222323242424242322D5
:102C000021201E1C1A181613110F0C0A080706059E
:102C10000404040507090C0F13181D23293038403C
:102C200048515A636D7780868D939AA0A7ADB3B94A
:102C3000BFC4CACFD4D9DDE1E5E9EDF0F2F5F7F98B
:102C4000FBFCFEFEFFFFFFFFFFFFFEFDFCFBF9F8B4
:102C5000F6F5F3F1EFEDECEAE8E6E5E3E2E0DFDEDE
:102C6000DDDCDBDBDADADADADADBDBDCDDDEDFE0A7
:102C7000E2E3E5E6E8EAECEDEFF1F3F5F6F8F9FB6F
:102C8000FCFDFEFFFFFFFFFFFFFEFEFCFBF9F7F57B
:102C9000F2F0EDE9E5E1DDD9D4CFCAC4BFB9B3ADF7
:102CA000A7A09A938D86807A736D666059534D47BD
:102CB000413C36312C27231F1B1713100E0B09071D
:102CC00005040202010100010101020304050708D5
:102CD0000A0B0D0F11131416181A1B1D1E2021228A
:102CE00023242525262626262625252423222120A1
:102CF0001E1D1B1A18161413110F0D0B0A080705B9
:102D00000403020101010001010202040507090B8D
:102D10000E1013171B1F23272C31363C41474D53F0
:102D20005960666D737A807E7C7A78767472706E84
:102D30006C6A68666462605E5C5A58565452504EC3
:102D40004C4A48464442403E3C3A38363432302EB3
:102D50002C2A28262422201E1C1A18161412100EA3
:102D60000C0A0806040200020406080A0C0E1012DF
:102D70001416181A1C1E20222426282A2C2E303223
:102D80003436383A3C3E40424446484A4C4E505213
:102D90005456585A5C5E60626466686A6C6E707203
:102DA0007476787A7C7E80828486888A8C8E9092F3
:102DB0009496989A9C9EA0A2A4A6A8AAACAEB0B2E3
:102DC000B4B6B8BABCBEC0C2C4C6C8CACCCED0D2D3
:102DD000D4D6D8DADCDEE0E2E4E6E8EAECEEF0F2C3
:102DE000F4F6F8FAFCFEFFFEFCFAF8F6F4F2F0EE68
:102DF000ECEAE8E6E4E2E0DEDCDAD8D6D4D2D0CE03
:102E0000CCCAC8C6C4C2C0BEBCBAB8B6B4B2B0AEF2
:102E1000ACAAA8A6A4A2A09E9C9A98969492908EE2
:102E20008C8A88868482807E7C7A78767472706ED2
:102E30006C6A68666462605E5C5A58565452504EC2
:102E40004C4A48464442403E3C3A38363432302EB2
:102E50002C2A28262422201E1C1A18161412100EA2
:102E60000C0A0806040201020406080A0C0E1012DD
:102E70001416181A1C1E20222426282A2C2E303222
:102E80003436383A3C3E40424446484A4C4E505212
:102E90005456585A5C5E60626466686A6C6E707202
:102EA0007476787A7C7E80828486888A8C8E9092F2
:102EB0009496989A9C9EA0A2A4A6A8AAACAEB0B2E2
:102EC000B4B6B8BABCBEC0C2C4C6C8CACCCED0D2D2
:102ED000D4D6D8DADCDEE0E2E4E6E8EAECEEF0F2C2
:102EE000F4F6F8FAFCFEFFFEFCFAF8F6F4F2F0EE67
:102EF000ECEAE8E6E4E2E0DEDCDAD8D6D4D2D0CE02
:102F0000CCCAC8C6C4C2C0BEBCBAB8B6B4B2B0AEF1
:102F1000ACAAA8A6A4A2A09E9C9A98969492908EE1
:102F20008C8A88868482807E7C7A78767472706ED1
:102F30006C6A68666462605E5C5A58565452504EC1
:102F40004C4A48464442403E3C3A38363432302EB1
:102F50002C2A28262422201E1C1A18161412100EA1
:102F60000C0A0806040201020406080A0C0E1012DC
:102F70001416181A1C1E20222426282A2C2E303221
:102F80003436383A3C3E40424446484A4C4E505211
:102F90005456585A5C5E60626466686A6C6E707201
:102FA0007476787A7C7E80828486888A8C8E9092F1
:102FB0009496989A9C9EA0A2A4A6A8AAACAEB0B2E1
:102FC000B4B6B8BABCBEC0C2C4C6C8CACCCED0D2D1
:102FD000D4D6D8DADCDEE0E2E4E6E8EAECEEF0F2C1
:102FE000F4F6F8FAFCFEFFFEFCFAF8F6F4F2F0EE66
:102FF000ECEAE8E6E4E2E0DEDCDAD8D6D4D2D0CE01
:10300000CCCAC8C6C4C2C0BEBCBAB8B6B4B2B0AEF0
:10301000ACAAA8A6A4A2A09E9C9A98969492908EE0
:103020008C8A88868482807E7C7A78767472706ED0
:103030006C6A68666462605E5C5A58565452504EC0
:103040004C4A48464442403E3C3A38363432302EB0
:103050002C2A28262422201E1C1A18161412100EA0
:103060000C0A0806040201020406080A0C0E1012DB
:103070001416181A1C1E20222426282A2C2E303220
:103080003436383A3C3E40424446484A4C4E505210
:103090005456585A5C5E60626466686A6C6E707200
:1030A0007476787A7C7E80828486888A8C8E9092F0
:1030B0009496989A9C9EA0A2A4A6A8AAACAEB0B2E0
:1030C000B4B6B8BABCBEC0C2C4C6C8CACCCED0D2D0
:1030D000D4D6D8DADCDEE0E2E4E6E8EAECEEF0F2C0
:1030E000F4F6F8FAFCFEFFFEFCFAF8F6F4F2F0EE65
:1030F000ECEAE8E6E4E2E0DEDCDAD8D6D4D2D0CE00
:10310000CCCAC8C6C4C2C0BEBCBAB8B6B4B2B0AEEF
:10311000ACAAA8A6A4A2A09E9C9A98969492908EDF
:103120008C8A88868482807E7D7A78767472706ECE
:103130006C6A68666462605E5C5A58565452504EBF
:103140004C4A48464442403E3C3A38363432302EAF
:103150002C2A28262422201E1C1A18161412100E9F
:103160000C0A0806040201020406080A0C0E1012DA
:103170001416181A1C1E20222426282A2C2E30321F
:103180003436383A3C3E40424446484A4C4E50520F
:103190005456585A5C5E60626466686A6C6E7072FF
:1031A0007476787A7D7E80828386888A8C8E9092EF
:1031B0009496989A9C9EA0A2A4A6A8AAACAEB0B2DF
:1031C000B4B6B8BABCBEC0C2C4C6C8CACCCED0D2CF
:1031D000D4D6D8DADCDEE0E2E4E6E8EAECEEF0F2BF
:1031E000F4F6F8FAFCFEFFFEFCFAF8F6F4F2F0EE64
:1031F000ECEAE8E6E4E2E0DEDCDAD8D6D4D2D0CEFF
:10320000CCCAC8C6C4C2C0BEBCBAB8B6B4B2B0AEEE
:10321000ACAAA8A6A4A2A09E9C9A98969492908EDE
:103220008C8A88868382807E7D7B78767572706ECC
:103230006C6A68666462605E5C5A58565452504EBE
:103240004C4A48464442403E3C3A38363432302EAE
:103250002C2A28262422201E1C1A18161412100E9E
:103260000C0A0807040201020407080A0C0E1012D7
:103270001416181A1C1E20222426282A2C2E30321E
:103280003436383A3C3E40424446484A4C4E50520E
:103290005456585A5C5E60626466686A6C6E7072FE
:1032A0007576787B7D7E80828385888A8B8E9092EE
:1032B0009496989A9C9EA0A2A4A6A8AAACAEB0B2DE
:1032C000B4B6B8BABCBEC0C2C4C6C8CACCCED0D2CE
:1032D000D4D6D8DADCDEE0E2E4E6E8EAECEEF0F2BE
:1032E000F4F6F8F9FCFEFFFEFCF9F8F6F4F2F0EE65
:1032F000ECEAE8E6E4E2E0DEDCDAD8D6D4D2D0CEFE
:10330000CCCAC8C6C4C2C0BEBCBAB8B6B4B2B0AEED
:10331000ACAAA8A6A4A2A09E9C9A98969492908EDD
:103320008B8A88858382807F7D7A78767473716ECC
:103330006C6A68676462605E5C5B58565452504EBB
:103340004C4A48464442403E3C3A38363432302EAD
:103350002C2A28262422211E1C1A18171512100E9A
:103360000C0B0906040202020406090B0C0E1012D3
:103370001517181A1C1E21222426282A2C2E30321A
:103380003436383A3C3E40424446484A4C4E50520D
:103390005456585B5C5E60626467686A6C6E7173F9
:1033A0007476787A7D7F80818386888A8C8D8F92EF
:1033B000949698999C9EA0A2A4A5A8AAACAEB0B2DF
:1033C000B4B6B8BABCBEC0C2C4C6C8CACCCED0D2CD
:1033D000D4D6D8DADCDEDFE2E4E6E8E9EBEEF0F2C0
:1033E000F4F5F7FAFCFEFEFEFCFAF7F5F4F2F0EE67
:1033F000EBE9E8E6E4E2DFDEDCDAD8D6D4D2D0CE00
:10340000CCCAC8C6C4C2C0BEBCBAB8B6B4B2B0AEEC
:10341000ACAAA8A5A4A2A09E9C99989694928F8DE0
:103420008C8A88868381807F7D7B79767472706ECA
:103430006D6B69676462605E5C5B59575552504EB4
:103440004C4A49474543403E3C3A38363533312EA5
:103450002C2A28262423211F1C1A18161413110F96
:103460000D0A0806040302030406080A0D0F1113CF
:103470001416181A1C1F21232426282A2C2E313317
:103480003536383A3C3E40434547494A4C4E505207
:103490005557595B5C5E60626467696B6D6E7072F4
:1034A0007476797B7D7F80818385878A8C8E9092EC
:1034B000939597999C9EA0A2A4A5A7A9ABAEB0B2E4
:1034C000B4B6B7B9BBBDC0C2C4C6C8CACBCDCFD2D3
:1034D000D4D6D8DADCDDDFE1E4E6E8EAECEDEFF1C2
:1034E000F3F6F8FAFCFDFEFDFCFAF8F6F3F1EFED69
:1034F000ECEAE8E6E4E1DFDDDCDAD8D6D4D2CFCD01
:10350000CBCAC8C6C4C2C0BDBBB9B7B6B4B2B0AEF0
:10351000ABA9A7A5A4A2A09E9C9997959392908EE3
:103520008C8A87858381807E7C7A78767472716FCD
:103530006D6B69676462605E5C5A58565553514FB3
:103540004D4B48464442403E3C3A39373533312FA3
:103550002C2A28262422201E1D1B19171513100E95
:103560000C09070604040304040607090C0E1013D3
:103570001517191B1D1E20222426282A2C2F313313
:103580003537393A3C3E40424446484B4D4F515303
:103590005556585A5C5E60626467696B6D6F7172F4
:1035A0007476787A7C7E80828486888A8C8E8F91ED
:1035B000939597999C9EA0A2A4A6A8AAABADAFB1E3
:1035C000B3B5B8BABCBEC0C2C4C6C7C9CBCDCFD1D3
:1035D000D4D6D8DADCDEE0E2E3E5E7E9EBEDF0F2C1
:1035E000F4F7F9FAFCFCFDFCFCFAF9F7F4F2F0ED63
:1035F000EBE9E7E5E3E2E0DEDCDAD8D6D4D1CFCD03
:10360000CBC9C7C6C4C2C0BEBCBAB8B5B3B1AFADF2
:10361000ABAAA8A6A4A2A09E9C99979593918F8EE1
:103620008C8A88868482807E7C7A78767472706ECA
:103630006C6A68676563615F5D5B59575553514EAE
:103640004C4A48464442403E3C3A38363533312FA6
:103650002D2B29272523211F1C1A181513110F0D97
:103660000B09080706060606060708090B0D0F11C9
:103670001315181A1C1F21232527292B2D2F313311
:103680003536383A3C3E40424446484A4C4E515307
:103690005557595B5D5F61636567686A6C6E7072F0
:1036A0007476787A7C7E80828486888A8C8E9092EA
:1036B000949698999B9D9FA1A3A5A7A9ABADAFB2E6
:1036C000B4B6B8BABCBEC0C2C4C6C8CACBCDCFD1CE
:1036D000D3D5D7D9DBDDDFE1E4E6E8EBEDEFF1F3BD
:1036E000F5F7F8F9FAFAFAFAFAF9F8F7F5F3F1EF6B
:1036F000EDEBE8E6E4E1DFDDDBD9D7D5D3D1CFCD03
:10370000CBCAC8C6C4C2C0BEBCBAB8B6B4B2AFADEC
:10371000ABA9A7A5A3A19F9D9B9998969492908EE3
:103720008C8A88868482807E7C7A787673716F6DCD
:103730006B6967656361605E5C5A585755535150B9
:103740004E4C4A48464442403E3C3A373533302E90
:103750002C29272522201E1C1917151412100F0DB5
:103760000C0B0A0A09090909090A0A0B0C0D0F10AA
:1037700012141517191C1E20222527292C2E303330
:1037800035373A3C3E40424446484A4C4E505153ED
:103790005557585A5C5E6061636567696B6D6F7100
:1037A0007376787A7C7E80828486888A8D8F9193E6
:1037B0009597999B9D9FA0A2A4A6A8A9ABADAFB0D9
:1037C000B2B4B6B8BABCBEC0C2C4C6C9CBCDD0D2E2
:1037D000D4D7D9DBDEE0E2E4E7E9EBECEEF0F1F39D
:1037E000F4F5F6F6F7F7F7F7F7F6F6F5F4F3F1F088
:1037F000EEECEBE9E7E4E2E0DEDBD9D7D4D2D0CDE2
:10380000CBC9C6C4C2C0BEBCBAB8B6B4B2B0AFAD04
:10381000ABA9A8A6A4A2A09F9D9B99979593918FD1
:103820008D8A88868482807F7D7B7A7876747371B6
:103830006F6D6B69676563615F5D5B59575452508B
:103840004D4B494644423F3D3A383633312F2C2ABE
:1038500028262422201E1C1A1917161413121110C0
:103860000F0F0E0E0D0D0D0D0D0E0E0F0F10111270
:1038700013141617191A1C1E20222426282A2C2F4E
:10388000313336383A3D3F424446494B4D5052540D
:1038900057595B5D5F61636567696B6D6F717374C9
:1038A00076787A7B7D7F8081838586888A8C8D8FF0
:1038B00091939597999B9D9FA1A3A5A7A9ACAEB005
:1038C000B3B5B7BABCBEC1C3C6C8CACDCFD1D4D6B2
:1038D000D8DADCDEE0E2E4E6E7E9EAECEDEEEFF090
:1038E000F1F1F2F2F3F3F3F3F3F2F2F1F1F0EFEEC0
:1038F000EDECEAE9E7E6E4E2E0DEDCDAD8D6D4D1C2
:10390000CFCDCAC8C6C3C1BEBCBAB7B5B3B0AEACE2
:10391000A9A7A5A3A19F9D9B99979593918F8D8C06
:063920008A888685838180
:00000001FF
